:020000040000FA
:1000000000008B012D28FF3F803120002000911E31
:100010000D28200090311F2080312100111E23283F
:1000200023002208230603191C282000111E2B2858
:100030009031472080312B28200023009E1C2B2844
:10004000210011122B2823002208230603192B2834
:10005000210011162B2820000900230000308C00FD
:1000600004308E00220000308C0000308E00210011
:100070000C308C0027308E00210018309900F001E0
:10008000F101F2017015240007308C0027000430C4
:100090008C002700083091002700003093002200D8
:1000A00000309D002100F3309E0020009A012000C6
:1000B000FF309B0020007F309C0021009F30950086
:1000C000200095012000ED010030CB002000A03081
:1000D000CE00CD003C30C6000030EC002000A03047
:1000E000D100D0000030C700993124218031220096
:1000F0008E15B1240130850022308400B824D03020
:10010000012500300125B824D13001257110D724F4
:1001100071148000CA24801BB4282200BE30A000C5
:10012000EF30A100B824D030012501300125B824DA
:10013000D13001257114D7241800D7241800D724F2
:100140001800D7241800D7241800D72418007110DD
:10015000D72471141800CA2410300006031DB428D7
:100160009031E4208031F22820000130A6070030D1
:10017000A73D031CBE28FF30A600A7002200DE30EA
:10018000A000AD30A1002000C801C901CA01223081
:10019000860001308700B824D030012500300125C9
:1001A00000301A00012500301A00012507301A001E
:1001B000012500301A00012507301A0001250430FE
:1001C0001A00012520301A00012510301A000125DF
:1001D000CA242000FF30B400B600B7000030B500DC
:1001E000B800B90022008E11B12491312F21803145
:1001F0002000931421001A30990070118B18542498
:100200000B186C24FF2381314C0E07390A3E03186A
:100210008A0A820014298329432B472B4B2B4F2B0F
:10022000000000000B24532B7115720803192029BC
:100230007111E4302924720829242030EA23F201C4
:1002400020004B0803192E297111D43029242000D5
:100250004B0829242030EA232000CB01711D82297C
:10026000701F7D29701320004B302202031D44298A
:1002700037302302031D442930302402031D442952
:100280003830250203194E2971114B30A200373046
:10029000A3003030A4003830A5007D2919309031FA
:1002A0000B208131B6301B0203301C3B031C7D291F
:1002B000200047080319542B4630292408304702F0
:1002C00003197A294C3029240830470203197A2966
:1002D000553029240830470203197A29533029243C
:1002E0000830470203197A29483029240830470288
:1002F000031D74292030EA2382299A310822813192
:10030000711D8229532B81316C086D070F398B3E8B
:1003100003188A0A8200BB29D029DB29F829032A7D
:10032000202A392A912AB12AC52AD52AF32A1B2B39
:100330002F2B000000000B24422B2A3084000130B8
:10034000850054081A0055081A0056081A00570864
:100350001A0058081A0008002A308400013085006D
:100360001200D4001200D5001200D6001200D700EF
:100370001200D800080020008E1DC02920003C106B
:1003800022008E1520009801FD3097008F309600D6
:10039000111000309900413098002000EC0A422BE7
:1003A0002000111CDA2920008E19D8292000BC1049
:1003B0002000EC0A422B20008E19E02920003C117D
:1003C000B82470300125E1300125083001250030C6
:1003D0000125CA2420009801FD3097008F30960037
:1003E000111000309900413098002000EC0A422B97
:1003F00020008E19FD292000BC112000111C022AAA
:100400002000EC0A422B20008E19082A20003C1202
:10041000B82470300125AC3001253330012500307F
:100420000125CA2420001030EE0020009C019D30E0
:100430009B009A01911005309C002000EC0A422B91
:1004400020008E19252A2000BC1220009118302A85
:1004500020006C08031DED000B241030EA23382A1D
:1004600020006C08031D372A6D08EC00ED01EC0A32
:10047000422B20008E193E2A20003C1320006C08DD
:10048000ED00B824713001257114D7242000C0007C
:10049000C01F762A7110D7247114CA246E1E532AE5
:1004A0003A0A031DBA0AEE033B086E026E08031CEB
:1004B000BB006E0803196F2A20009801FF309700D7
:1004C000D9309600111000309900413098000B246B
:1004D0002000ED010530EC001030EA23902A2200C4
:1004E0008E11B1240B242000ED01902AD724200086
:1004F000C100D7242000C200D7242000C300D72485
:100500002000C4007110D72471142000C500CA2433
:1005100022008E11B1242000ED0A0B241030EA23B2
:10052000422B20008E1D962A2000BC132000450877
:10053000D4004408D50043080F39D600D701D801AC
:100540002030D9004E30DA00DB01DC01DD019031D2
:100550006B2082319D212000ED0A0B241030EA230C
:10056000422BAC2120000030D9000030DA001030DE
:10057000DB00DC01DD019031992082319D212000DA
:10058000ED0A0B241030EA23422BAC2120008830E6
:10059000D9001330DA00DB01DC01DD019D212000F0
:1005A000ED0A0B241030EA23422BAC212000540822
:1005B000BE0036025508BF00373B031CE32A54082F
:1005C000B6005508B700540838025508393B0318DF
:1005D000ED2A5408B8005508B9002000ED0A0B2494
:1005E0001030EA23422B20004308D4004208D500F3
:1005F0004108D600D60CD50CD40CD60CD50CD40C96
:10060000D60CD50CD40CD60CD50CD40C0F30D6058A
:10061000D701D8016430D9000030DA00DB01DC01F9
:10062000DD0190316B2083319D212000ED0A0B24E8
:100630001030EA23422BAC2120000030D9000030DA
:10064000DA001030DB00DC01DD01903199208331CC
:100650009D212000ED0A0B241030EA23422BAC210F
:1006600020005408BD003402031C382B5408B40089
:100670005408350203183E2B5408B5000B24200003
:10068000ED01422B532B883100208331532B8831CD
:10069000F7208331532B89312B218331532B89311F
:1006A000D7218331532BFE28210018309900701573
:1006B00022000E1623006D30A200A3002300463056
:1006C000A000A100230047309B0000309C000830B0
:1006D0009F0026309E0090309D0021007112F11283
:1006E0009116C0308B00983100208331772B2A255A
:1006F000031863258B1C7F2B8B107017772B701FB3
:100700008C2B7013193090310B208331B6301B02C3
:1007100003301C3B031C8D2B772B230000309D00E6
:1007200022000E128B01711EA02B711220000130CD
:10073000A8070030A93D031CA02BFF30A800A9008A
:1007400098310020833122008E15B12401308500BC
:1007500022308400B824D030012500300125B8248F
:10076000D13001257114D7241A00D7241A00D724B8
:100770001A00D7241A00D7241A00D7241A00D72425
:100780001A007110D72471148000CA24103000069A
:100790000319D22BB824D0300125073001251030A1
:1007A0000125CA2422008E119031E4208331F11EEC
:1007B000E22BF1122200FE30A000ED30A1009131B9
:1007C0002F21833121001A30990070112700003049
:1007D0009300FE282000CC004608031DF12BF214E4
:1007E000FE2B023085004E0884004C081A000408D5
:1007F000DC3A03197C30DC3ACE00C6030800200046
:100800003C3046020319092C023085004D08840053
:100810000008CC00080020003C304602031D122CCA
:100820007214202C023085004D0884004D0ADC3AF9
:1008300003197C30DC3ACD00C60AEC010008CC007C
:100840000800CC00023085004D0884004C08800070
:1008500008002000CF003C304702031C312CF21569
:100860003E2C00308500510884004F081A0004080F
:10087000DC3A03197C30DC3AD100C70A08002000BA
:100880004708031D452C7215532C00308500500875
:1008900084001200CF000408DC3A03197C30DC3AF3
:1008A000D000C7034F0808008B10701720000130DC
:1008B000C807031C612C1030EA230030C93D00300A
:1008C000CA3D803048025130493B01304A3B031C4D
:1008D0006B2C4030EA2308002700003093002000F2
:1008E000931C9A2C28009701D930960095019310FB
:1008F0004430970020000130B1070030B23D003095
:10090000B33D031C872CFF30B100B200B3003E3072
:100910004702033E031C8F2C4B0FCB0A9A2C4A082C
:10092000C630031DC7302924490829244808292432
:100930002030EA23200008002300910095131513AE
:1009400015141308200008002300930095131513B5
:10095000151555309600AA309600951415112000F3
:100960000800701DB72C0E30F600F60BB52C0800F1
:1009700021008E14B12422000E14B12422008E1006
:1009800021008E10B12422000E1021000E10B1247F
:100990002000080022008E1021008E10B1242100BA
:1009A0000E14B12421008E14B1242000080021006F
:1009B0008E140830F7000310F80D22000E142000EA
:1009C0000E1CDF2CB12420008E18781422000E108B
:1009D00021000E10B124F70BDB2C22008E10210019
:1009E00071188E10711C8E1421000E14B124220077
:1009F0000E1021000E10B12421008E147808200062
:100A00000800F8000830F70002308E10F81B092D9E
:100A10000C2D21008E140F2D21008E100F2DB124CE
:100A200021000E14B124F80D22000E1021000E102A
:100A3000B124F70B042D21008E14B1240E14B1241F
:100A4000F1148E1CF11022000E1021000E10B124A2
:100A500020000800230020082106031D03140319A9
:100A600003100319462D382D200821060319342DB3
:100A700002308500200884000008A600200A473ABA
:100A800003196730473AA000260803142000080025
:100A90002108A00008002300A700023085002308D9
:100AA0008400013E6E3A031929306E3AA4002206F2
:100AB0000319602D270880002408A30021001116C7
:100AC0002708200008002300AB0024302B06031960
:100AD000AC0185312C080F39703E03188A0A820058
:100AE000802D8A2DB42DD32DFC2D122F122F122FD5
:100AF000122F122F122F122F122F122F122F122FEE
:100B000001308500AE3084002B088000F0110130E8
:100B1000AC00162F01308500AF3084002B08800018
:100B2000AD00AD1F942D122FB030AA0085312D0ECF
:100B300003399D3E03188A0A8200A42DA42DA12DFD
:100B4000A72D0030A900B12D0130A900AA2D033036
:100B5000A900AA2D2D1BB02D2D080F39013EA90784
:100B6000B12D0230AC00162F2908031DBA2D033019
:100B7000AC00692DF01DC02DF0112F30AB02C62D39
:100B80002F302B02031DC62DF015D22D013085000C
:100B90002A0884002B081A000408AA00A90BD22DE9
:100BA0000330AC00162FF01DD92DF0112F30AB0201
:100BB000DF2D2F302B02031DDF2DF015FB2D013013
:100BC00085002A0884002B0880000030F900AE3030
:100BD0002A02A900A90301308500AF308400120069
:100BE000F907A90BEF2D7909013E0002031D122F11
:100BF0000430AC00692D162F711601308500AF301E
:100C0000840000080F39013EA9008631000E033927
:100C10000C3E03188A0A8200102E572EB82ED62EAC
:100C200022008E1523000008AD00B124013085009C
:100C3000B0308400B824D03001251200DE00012538
:100C400023002D1B3D2E1200DF005E08003A031D1D
:100C50002C2E7F30DF05332E073A031D322E103045
:100C6000DF00332E332EDE0A5F0801252300A90B97
:100C7000232ECA241A27F116112F2330AE00290380
:100C80009038AF0001308500B0308400B824D130F6
:100C900001257114D7241A002300A90B492E7110C5
:100CA000D724CA2422008E11B1242127112F01300C
:100CB0008500B0308400801F5E2E8C2E00308700AF
:100CC00020308600120086070318870A2F1B7D2E0E
:100CD000230022300602031C712E3D300602031C45
:100CE000742E12001600762E12001E00A90B692E1B
:100CF0009831002086311A27112F2330AE002903A6
:100D00009038AF0001308500B030840016001A0022
:100D1000A90B862E2127112F1200230091002F1BD3
:100D2000A52E951315131515120093008B1355302E
:100D30009600AA30960095148B1795189D2E910A4F
:100D4000A90B942E15111A27112F2330AE00290359
:100D50009038AF0001308500B03084009513151332
:100D6000151413081A00910AA90BB02E2127112F70
:100D7000863100080F39BF3E03188A0A8200D02E40
:100D8000D02ECF2ED02ED02ED42ED02ED02ED12E6F
:100D9000D22ED32ED02ED02ED02ED02ED02E112F1C
:100DA000112F112F112F112F1A27112F230012008D
:100DB000AD0020001200EB001200EA001200E90072
:100DC00023002D1BFE2E22008E15B124B8242000F6
:100DD0006B0D0E39A03801256A0801256908012527
:100DE000120001252300A90BF02ECA249031002007
:100DF000863122008E11B1241A27112F23002330AF
:100E0000AE0029039038AF0001308500B030840077
:100E1000662777271A002300A90B092F7A27212795
:100E2000112F122F2300AC014825162F2A25031855
:100E3000632D080023304B258A304B2576304B2517
:100E4000080001308500AF3084002300A9012F0E77
:100E500007390319322FAA002F080F39013EA907BD
:100E6000AA0B2F2F013EA9000030F9001200F9074C
:100E7000A90B362F7909013E1A000408AA00013097
:100E80008700AE3086007016F011F01D4B2FF01168
:100E900016002F3E5F2F701A5D2F233001020319B9
:100EA000592F243001020319592F2F300102031D3D
:100EB0005D2FF0152F304B25452F701216004B2556
:100EC000060823002A02031D452F080022008E1564
:100ED000B124B82420006B0D0E39A03801256A0812
:100EE000012569080125B824A930012508007114DD
:100EF000D72408007110D7247114CA2422008E113F
:100F0000B1240800FF3FFF3FFF3FFF3FFF3FFF3F90
:100F1000FF3FFF3FFF3FFF3FFF3FFF3FFF3FFF3FE1
:100F2000FF3FFF3FFF3FFF3FFF3FFF3FFF3FFF3FD1
:100F3000FF3FFF3FFF3FFF3FFF3FFF3FFF3FFF3FC1
:100F4000FF3FFF3FFF3FFF3FFF3FFF3FFF3FFF3FB1
:100F5000FF3FFF3FFF3FFF3FFF3FFF3FFF3FFF3FA1
:100F6000FF3FFF3FFF3FFF3FFF3FFF3FFF3FFF3F91
:100F7000FF3FFF3FFF3FFF3FFF3FFF3FFF3FFF3F81
:100F8000FF3FFF3FFF3FFF3FFF3FFF3FFF3FFF3F71
:100F9000FF3FFF3FFF3FFF3FFF3FFF3FFF3FFF3F61
:100FA000FF3FFF3FFF3FFF3FFF3FFF3FFF3FFF3F51
:100FB000FF3FFF3FFF3FFF3FFF3FFF3FFF3FFF3F41
:100FC000FF3FFF3FFF3FFF3FFF3FFF3FFF3FFF3F31
:100FD000FF3FFF3FFF3FFF3FFF3FFF3FFF3FFF3F21
:100FE000FF3FFF3FFF3FFF3FFF3FFF3FFF3FFF3F11
:100FF000FF3FFF3FFF3FFF3FFF3FFF3FFF3FFF3F01
:1010000088316C080739073E03188A0A82001328C2
:101010001E2831283728C128000000000000843134
:101020000B248831F6282000EC0A20000830470203
:1010300003181D2884310B248831F62822007010F3
:101040008E1970148E1520009801FF309700E03043
:101050009600111000309900413098002000EC0AF1
:10106000F6282000111C36282000EC0AF62807304C
:101070002E05031945280830AE070030AF3D00307B
:10108000B03D0730FF3AAE05721604303002031C43
:101090004D2806303002031C57280030AE00AB004C
:1010A0000030AF00AC000430B000AD00F2160430E8
:1010B0002D02031C5F2806302D02031C66282E0813
:1010C000AB002F08AC003008AD0072172E082B02C1
:1010D000D4002F082C3BD50030082D3BD600031C34
:1010E000952803199528D409D509D6090130D407C4
:1010F0000030D53D0030D63D083054020318952805
:101100005508031D95285608031D9528F217013030
:10111000AC070030AD3D06302D02031C9528003091
:10112000AB000130AC000430AD008431B82488310C
:10113000300D0E39A0388531012588312F088531D1
:10114000012588312E088531012588310830FA00C3
:1011500084313F248831853101258831FA0BA82854
:101160008431CA24883120009801FF30970038303C
:101170009600111000309900413098002000EC0AD0
:10118000F6282000111CF5280830AE070030AF3DCE
:101190000030B03D06303002031CE3280030AE00C2
:1011A0000030AF000430B0002E082B022F082C3B7B
:1011B00030082D3B031DE3280030AB000130AC00AC
:1011C0000430AD00F2172000083047020318F2285F
:1011D0002200701C8E118431B124883184310B249B
:1011E0008831F52820000330EC00F628080088310B
:1011F0006C080339FE3E03188A0A820006290C296E
:101200002229000084310B2489312A2923009518D2
:101210000B292000EC0A2A2984310B2489318431DE
:101220000B248931230091008331FF2389318431DC
:10123000A424893120000230EC0030308431212494
:1012400089312A2923009518292984310B248931D1
:10125000F0172A29080089316C080F39323E03182B
:101260008A0A8200462959295F297A299E29A929B3
:10127000AF29B529BB2900000000000000000000D4
:101280000000000084310B248931D629220070101F
:101290008E1970148E1520009801FF309700E030F1
:1012A0009600111000309900413098002000EC0A9F
:1012B000D6292000111C5E292000EC0AD629843191
:1012C000B8248931D030853101258931003085310C
:1012D000012589318431B8248931D1308531012506
:1012E000893171148431D72489312200A200200071
:1012F000EC0AD62901308500233084008431D724BC
:1013000089311A008431D72489311A008431D724D5
:1013100089311A008431D72489311A008431D724C5
:1013200089311A0071108431D724893171141A005F
:101330008431CA2489312000EC0AD6292200FA30EF
:10134000A000CE30A10091312F2189312000EC0A7C
:10135000D6299031E82089312000EC0AD629913134
:10136000072189312000EC0AD629913120218931C9
:101370002000EC0AD6292000FF30B400B600B700E8
:101380000030B500B800B90010308331EA2389314C
:101390002200701C8E118431B124893184310B24D8
:1013A000893150308331EA238931D62908008931C7
:1013B0006C080339DE3E03188A0A8200E629F62902
:1013C000042A3A2A84310B248931422A02300E162B
:1013D00020009801F3309700CB30960011100030B8
:1013E0009900413098002000EC0A422A2000111C8C
:1013F000032A210019309D00220081309700171F19
:10140000FF292000EC0A422A21009D149D18062A7B
:101410009D0122000030970002300E122100B630EC
:101420001B0203301C3B03182C2A1B082000D4008D
:1014300021001C082000D50020000310D50CD40C7E
:10144000B430D4020030D53B031C2C2A5508FF30A1
:10145000031DD4005408AA0020009801F33097001F
:10146000CB309600111000309900413098002000D8
:10147000EC0A422A2000111C412A84310B248A31B3
:10148000412A422A0800FF3FFF3FFF3FFF3FFF3F47
:10149000FF3FFF3FFF3FFF3FFF3FFF3FFF3FFF3F5C
:1014A000FF3FFF3FFF3FFF3FFF3FFF3FFF3FFF3F4C
:1014B000FF3FFF3FFF3FFF3FFF3FFF3FFF3FFF3F3C
:1014C000FF3FFF3FFF3FFF3FFF3FFF3FFF3FFF3F2C
:10200000701D0A281430F4000030F500F50B062886
:10201000F40B0628080021009D0022008130970063
:10202000171F10288431B124903121009D149D1870
:1020300017289D0122000030970021000800F010B1
:1020400023009D1C2A28F0141D121D1A24281D1679
:102050001D1E27281D1D2E28F0141908F0184328CE
:102060001908A500210A473A03196730473AA80022
:102070002002031943282108840002308500250826
:1020800080002808A1002000911A1F2808002300C2
:10209000023085002208840012009A0004086E3A7B
:1020A000031929306E3AA20008005908D4075A08CB
:1020B000D53D5B08D63D5C08D73D5D08D83D08009E
:1020C0005908D4025A08D53B5B08D63B5C08D73B7D
:1020D0005D08D83B0800D210D2115408DE00550824
:1020E000DF005608E0005708E1005808E200D4017C
:1020F000D501D601D701D8012830D300E20CE10C7C
:10210000E00CDF0CDE0C5215D21D5211031C5211D3
:102110005219D214031855200318D2140310D90DE4
:10212000DA0DDB0DDC0DDD0D0318D215D30B7E2887
:102130000800D21059085A045B045C045D040319BA
:10214000D2145408DE005508DF005608E000570896
:10215000E1005808E200D401D501D601D701D80129
:102160002830D300DE0DDF0DE00DE10DE20DD40DC2
:10217000D50DD60DD70DD80D60205216031C521266
:10218000031C55200314521E0310D30BB228DE0D7E
:10219000DF0DE00DE10DE20D5E08D4005F08D50013
:1021A0006008D6006108D7006208D8000800540E05
:1021B0000F39D5000F30D40555080319E3280A302C
:1021C000D407D503DC280800E820072120210800D7
:1021D000220024082000D400D72007305402F93010
:1021E000031C1130D407D501D601D701D801103016
:1021F000D9000E30DA00DB01DC01DD016B202000AC
:102200005408C8005508C9005608CA000800220032
:1022100023082000D400D720D501D601D701D8014A
:102220003C30D9000030DA00DB01DC01DD016B203D
:1022300020005408C8075508C93D5608CA3D080083
:10224000220022082000D400D720D501D60120008A
:102250005408C8075508C93D5608CA3D0800A630AD
:10226000F90084312924913122002008F9078431B2
:102270002924913122002108F90784312924913140
:1022800028308600013087001700F907843129249F
:1022900091311700F9078431292491311700F9078A
:1022A00084312924913117001700F907843129243A
:1022B00091311700F9078431292491311700F9076A
:1022C0008431292491313130860000308700160096
:1022D000F9078431292491311600F9078431292422
:1022E00091311600F9078431292491311600F9073C
:1022F0008431292491311600F90784312924913140
:102300001600F9078431292491311600F907843128
:10231000292491311600F9078431292491311600BE
:10232000F9078431292491317909013E8431292426
:10233000913120308331EA2391310800FF3FFF3F84
:10234000FF3FFF3FFF3FFF3FFF3FFF3FFF3FFF3F9D
:10235000FF3FFF3FFF3FFF3FFF3FFF3FFF3FFF3F8D
:10236000FF3FFF3FFF3FFF3FFF3FFF3FFF3FFF3F7D
:10237000FF3FFF3FFF3FFF3FFF3FFF3FFF3FFF3F6D
:103000002300DD010030E7215A3A230003190C2880
:10301000FF3A0319132801004030D6000030D700D2
:10302000A530D9001A280030D6004030D7005A30D9
:10303000D9001A28230002305607E721220203197B
:1030400023282208F121230003305607E721230219
:1030500003192C282308F121230004305607E72107
:103060002402031935282408F121230005305607CE
:10307000E721250203193E282508F1212300063007
:103080005607E7212602031947282608F1212300C5
:1030900007305607E7212702031950282708F12196
:1030A000230008305607E721280203195928280869
:1030B000F121230009305607E7212902031962286C
:1030C0002908F12123000A305607E7212A020319B3
:1030D0006B282A08F12123000B305607E7212B0229
:1030E000031974282B08F12123000C305607E7211F
:1030F0002C0203197D282C08F12123000D305607DE
:10310000E7212D02031986282D08F12123000E3016
:103110005607E7212E0203198F282E08F1212300DC
:103120000F305607E7212F02031998282F08F121A5
:10313000230010305607E72130020319A128300878
:10314000F121230011305607E72131020319AA2883
:103150003108F121230012305607E721320203190A
:10316000B3283208F121230013305607E721330238
:103170000319BC283308F121230014305607E72136
:1031800034020319C5283408F121230015305607ED
:10319000E72135020319CE283508F1212300163026
:1031A0005607E72136020319D7283608F1212300F4
:1031B00017305607E72137020319E0283708F121B5
:1031C000230018305607E72138020319E928380888
:1031D000F121230019305607E72139020319F2289B
:1031E0003908F12123001A305607E7213A02031962
:1031F000FB283A08F12123001B305607E7213B0248
:10320000031904293B08F12123001C305607E7214C
:103210003C0203190D293C08F12101302300570716
:10322000E7212300D80001305607E7212300D80A00
:10323000FF3058060319D80A5808F1210030E72159
:1032400023005908F12108002300DD010030E721A7
:1032500023005A3A03195529FF3A03195729013017
:10326000E7212300DB000130403EE7212300DC00A2
:10327000FF305B0603195729FF305C0603195529F7
:10328000FE305B0603195129FE305C0603194D29F7
:103290005B085C02031C552957295B08031D57294D
:1032A00055295C08031D55295729003059294030FC
:1032B0005929DA00023023005A07E721A200023020
:1032C00023005A07E721A200033023005A07E72111
:1032D000A300043023005A07E721A400053023008F
:1032E0005A07E721A500063023005A07E721A60068
:1032F000073023005A07E721A700083023005A07A8
:10330000E721A800093023005A07E721A9000A3065
:1033100023005A07E721AA000B3023005A07E721B0
:10332000AB000C3023005A07E721AC000D3023001E
:103330005A07E721AD000E3023005A07E721AE00FF
:103340000F3023005A07E721AF00103023005A073F
:10335000E721B000113023005A07E721B1001230F5
:1033600023005A07E721B200133023005A07E72150
:10337000B300143023005A07E721B40015302300AE
:103380005A07E721B500163023005A07E721B60097
:10339000173023005A07E721B700183023005A07D7
:1033A000E721B800193023005A07E721B9001A3085
:1033B00023005A07E721BA001B3023005A07E721F0
:1033C000BB001C3023005A07E721BC000800230083
:1033D0009518E8299100951315131514130820006A
:1033E000080023009518F22993009513151315155D
:1033F000F0128B1BF0168B1355309600AA309600F6
:103400009514F01E8B13F01A8B171511200008006D
:103410002230840085011B30FA00003084319C2466
:103420009A315A3A0319182AFF3A03191A2A010045
:1034300040301C2A00301C2A230091009A315D087C
:103440000339253E03188A0A8200292A4C2A6D2A4C
:10345000832A2300023091079513151315141200C7
:1034600013020319442A1100860030308331EA2305
:103470009A31230011088331EA239A3106088331F7
:10348000EA239A317111862A910AFA0B2E2AF01F2B
:103490004B2ADD0A7111862A01301107403A91004A
:1034A0009513151315141308013E9300FF301306EE
:1034B0000319930A30308331EA239A31230011082B
:1034C000403A8331EA239A31230013088331EA23F7
:1034D0009A312300DD0A7111862A1108A5300319DB
:1034E0005A30930030308331EA239A3100308331EF
:1034F000EA239A31230013088331EA239A31230007
:10350000DD0A7111862AF013DD01862A20000800E9
:10351000270000309300013087000E3086008119AB
:10352000922A942A8111FE288115FE28E501E601E0
:10353000E701E800E830E3020330E43B031CA22A81
:10354000E50A9A2AE830E3070330E43D6430E302F9
:103550000030E43B031CAE2AE60AA62A6430E307E7
:103560000030E43D0A30E70AE3020318B32AE70318
:103570006307E8000800FF3FFF3FFF3FFF3FFF3FBB
:10358000FF3FFF3FFF3FFF3FFF3FFF3FFF3FFF3F4B
:10359000FF3FFF3FFF3FFF3FFF3FFF3FFF3FFF3F3B
:1035A000FF3FFF3FFF3FFF3FFF3FFF3FFF3FFF3F2B
:1035B000FF3FFF3FFF3FFF3FFF3FFF3FFF3FFF3F1B
:020000040001F9
:10E000005A0063004B003700300038000000000069
:10E0100000000000AA000000000004000000000052
:10E020000400000000000000FF000000FF00FF00EF
:10E03000000000000000FF00FF00FF00FF00FF00E5
:10E04000FF00FF00FF00FF00FF00FF00FF00FF00D8
:10E05000FF00FF00FF00FF00FF00FF00FF00FF00C8
:10E06000FF00FF00FF00FF00FF00FF00FF00FF00B8
:10E07000FF00FF00FF00FF00FF00FF00FF00FF00A8
:10E080005A006200FF00FF00FF00FF00FF00FF00DA
:10E09000FF00FF00FF00FF00FF00FF00FF00FF0088
:10E0A000FF00FF00FF00FF00FF00FF00FF00FF0078
:10E0B000FF00FF00FF00FF00FF00FF00FF00FF0068
:10E0C000FF00FF00FF00FF00FF00FF00FF00FF0058
:10E0D000FF00FF00FF00FF00FF00FF00FF00FF0048
:10E0E000FF00FF00FF00FF00FF00FF00FF00FF0038
:10E0F000FF00FF00FF00FF00FF00FF00FF00FF0028
:10E1000041005000500020005300430052004100E5
:10E11000540043004800500041004400FF00FF004D
:10E12000FF00FF00FF00FF00FF00FF00FF00FF00F7
:10E13000FF00FF00FF00FF00FF00FF00FF00FF00E7
:10E14000FF00FF00FF00FF00FF00FF00FF00FF00D7
:10E15000FF00FF00FF00FF00FF00FF00FF00FF00C7
:10E16000FF00FF00FF00FF00FF00FF00FF00FF00B7
:10E17000FF00FF00FF00FF00FF00FF00FF00FF00A7
:10E18000FF00FF00FF00FF00FF00FF00FF00FF0097
:10E19000FF00FF00FF00FF00FF00FF00FF00FF0087
:10E1A000FF00FF00FF00FF00FF00FF00FF00FF0077
:10E1B000FF00FF00FF00FF00FF00FF00FF00FF0067
:10E1C000FF00FF00FF00FF00FF00FF00FF00FF0057
:10E1D000FF00FF00FF00FF00FF00FF00FF00FF0047
:10E1E000FF00FF00FF00FF00FF00FF00FF00FF0037
:10E1F000FF00FF00FF00FF00FF00FF00FF00FF0027
:04000E00020FFC1CC5
:08000000FF3FFF3FFF3FFF3F00
:00000001FF
